:020000040800F2
:10100000003C002071410008B94100081D4E000855
:10101000214E0008254E0008294E0008000000005F
:101020000000000000000000000000002D4E00083D
:10103000314E000800000000354E0008394E00080F
:10104000B9410008B9410008B9410008B941000898
:10105000B9410008B9410008B9410008DD4F000856
:10106000000000003D4E0008654E0008A14E00083B
:10107000514F0008B9410008B941000800000000C4
:10108000B94F0008B941000800000000814F000876
:10109000A14F0008914F0008B9410008B94100086C
:1010A000B9410008B9410008B9410008B54F00082E
:1010B000B94100080000000000000000000000002E
:0C10C000B941000800000000B941000820
:1010CC004FF0FF0C1CEAD0521EBF1CEAD15392EA1F
:1010DC000C0F93EA0C0F6FD01A4480EA010C4002FB
:1010EC0018BF5FEA41211ED04FF0006343EA501055
:1010FC0043EA5111A0FB01310CF00040B1F5000F97
:10110C003EBF490041EAD3715B0040EA010062F145
:10111C007F02FD2A1DD8B3F1004F40EBC25008BF2F
:10112C0020F00100704790F0000F0CF0004C08BF4D
:10113C0049024CEA502040EA51207F3AC2BFD2F11A
:10114C00FF0340EAC250704740F400004FF0000328
:10115C00013A5DDC12F1190FDCBF00F00040704762
:10116C00C2F10002410021FA02F1C2F1200200FAA0
:10117C0002FC5FEA310040F1000053EA4C0308BF67
:10118C0020EADC70704792F0000F00F0004C02BFB8
:10119C00400010F4000F013AF9D040EA0C0093F033
:1011AC00000F01F0004C02BF490011F4000F013B8D
:1011BC00F9D041EA0C018FE70CEAD15392EA0C0FFB
:1011CC0018BF93EA0C0F0AD030F0004C18BF31F066
:1011DC00004CD8D180EA010000F00040704790F03C
:1011EC00000F17BF90F0004F084691F0000F91F0E0
:1011FC00004F14D092EA0C0F01D142020FD193EAA6
:10120C000C0F03D14B0218BF084608D180EA01002D
:10121C0000F0004040F0FE4040F40000704740F009
:10122C00FE4040F44000704780F0004002E000BFF8
:10123C0081F0004142001FBF5FEA410392EA030FB5
:10124C007FEA226C7FEA236C6AD04FEA1262D2EBFF
:10125C001363C1BFD218414048404140B8BF5B4204
:10126C00192B88BF704710F0004F40F4000020F09D
:10127C007F4018BF404211F0004F41F4000121F0B3
:10128C007F4118BF494292EA030F3FD0A2F10102FD
:10129C0041FA03FC10EB0C00C3F1200301FA03F13B
:1012AC0000F0004302D5494260EB4000B0F5000F5E
:1012BC0013D3B0F1807F06D340084FEA310102F11D
:1012CC000102FE2A51D2B1F1004F40EBC25008BFCF
:1012DC0020F0010040EA03007047490040EB000099
:1012EC00013A28BFB0F5000FEDD2B0FA80FCACF19A
:1012FC00080CB2EB0C0200FA0CF0AABF00EBC250C7
:10130C0052421843BCBFD0401843704792F0000FB4
:10131C0081F4000106BF80F400000132013BB5E707
:10132C004FEA41037FEA226C18BF7FEA236C21D07D
:10133C0092EA030F04D092F0000F08BF08467047E2
:10134C0090EA010F1CBF0020704712F07F4F04D1B0
:10135C00400028BF40F00040704712F100723CBFC3
:10136C0000F50000704700F0004343F0FE4040F4ED
:10137C00000070477FEA226216BF08467FEA2363AB
:10138C000146420206BF5FEA412390EA010F40F496
:10139C00800070474FF0000304E000BF10F00043E2
:1013AC0048BF40425FEA000C08BF704743F09643C9
:1013BC0001464FF000001CE050EA010208BF7047E4
:1013CC004FF000030AE000BF50EA010208BF70476B
:1013DC0011F0004302D5404261EB41015FEA010C80
:1013EC0002BF84460146002043F0B64308BFA3F178
:1013FC008053A3F50003BCFA8CF2083AA3EBC2535A
:10140C0010DB01FA02FC634400FA02FCC2F1200278
:10141C00BCF1004F20FA02F243EB020008BF20F0AF
:10142C000100704702F1200201FA02FCC2F1200215
:10143C0050EA4C0021FA02F243EB020008BF20EA0A
:10144C00DC7070474FF0FF3C06E000BF4FF0010C22
:10145C0002E000BF4FF0010C4DF804CD4FEA400202
:10146C004FEA41037FEA226C18BF7FEA236C11D04C
:10147C0001B052EA530C18BF90EA010F58BFB2EBFF
:10148C00030088BFC81738BF6FEAE17018BF40F07F
:10149C00010070477FEA226C02D15FEA402C05D133
:1014AC007FEA236CE4D15FEA412CE1D05DF8040BB8
:1014BC00704700BF844608466146FFE70FB5FFF74B
:1014CC00C9FF002848BF10F1000F0FBD4DF808ED03
:1014DC00FFF7F4FF0CBF012000205DF808FB00BFF4
:1014EC004DF808EDFFF7EAFF34BF012000205DF84E
:1014FC0008FB00BF4DF808EDFFF7E0FF94BF01209B
:10150C0000205DF808FB00BF4DF808EDFFF7D2FF97
:10151C0094BF012000205DF808FB00BF4DF808EDDA
:10152C00FFF7C8FF34BF012000205DF808FB00BFA7
:10153C004FEA4002B2F1FE4F0FD34FF09E03B3EBD4
:10154C0012620DD94FEA002343F0004310F0004F14
:10155C0023FA02F018BF404270474FF0000070476A
:10156C0012F1610F01D1420205D110F0004008BF09
:10157C006FF0004070474FF00000704742000ED2F1
:10158C00B2F1FE4F0BD34FF09E03B3EB126209D4B2
:10159C004FEA002343F0004323FA02F070474FF068
:1015AC000000704712F1610F01D1420202D14FF0DD
:1015BC00FF3070474FF00000704700BF53B94AB975
:1015CC00002908BF00281CBF4FF0FF314FF0FF303F
:1015DC0000F00CB8ADF1080C6DE904CE04F014FC6D
:1015EC00DDF804E0DDE9022304B07047704700BF6A
:1015FC0010B5054C237833B9044B13B10448AFF341
:10160C0000800123237010BD6E0800200000000034
:10161C003C61000808B5034B1BB103490348AFF309
:10162C00008008BD00000000700800203C6100082C
:10163C00A449A5480B68CA6F00882DE9F04FD21A4F
:10164C0092B2A24C5509904283B02280658062D23E
:10165C009F48008890425ED99E480022028004F187
:10166C004006204601E051F8083F4A68D21A92B26F
:10167C0095422CBF0022012240F8042F8642F2D161
:10168C00A56BA368D4F818A0D4F804E06169A26A29
:10169C00D4F824B02069D4F820800193AE00656B97
:1016AC00E768D4F82CC083EA0A0946EAC50689EA39
:1016BC0002098EEA010585EA0B054FEA8909E369FF
:1016CC00009349EAC509256C236B354380EA08066B
:1016DC005E4049EA0609E66B009B45EA4605EEB218
:1016EC0087EA03057C4B85EA0C0549EA450593F826
:1016FC000090EDB2B9F1000F10D0DFF8E09199F83D
:10170C000090B9F1000F0FD1AE4211D0B4F85030A7
:10171C000133A4F8503003B0BDE8F08FDFF8BC9172
:10172C0099F80030002B60D0C6F10F06F6B2EBE74B
:10173C00684BB4F8465000261E80019B5B0243EABE
:10174C008E2343EA0C0343EA072343EAC013013513
:10175C0043EA81130099A4F8465043EA4A13256BD7
:10176C0043EA0113012D43EAC80308BF5C4E43EA68
:10177C008B0343EA420208BF35702F2A1BDD94F815
:10178C004830002B5BD1574D2A78002AC3D0564BDA
:10179C001B78002BBFD1504B1B78002BBBD094F87F
:1017AC004B30934253D0042A84F84B205AD901234E
:1017BC0084F84930AFE7531E2E2B0FD9002AE2D103
:1017CC0094F84A304949012B08BF84F84820454A0F
:1017DC0000230B80137084F849309CE7434B414D38
:1017EC000021D2B219802A70D1E703F01DFDC0B1DF
:1017FC0094F844300133DBB2642B84F8443010D9B4
:10180C00012389F80030D4E901E30193E3690093E3
:10181C00D4E90370D4E9051AD4E9088BD4E90A2C6D
:10182C0082E7D4E901E30193E3690093D4E90370FF
:10183C00D4E9051AD4E9088BD4E90A2C5FE72B48C4
:10184C002849028000230B7084F8493063E7042A8E
:10185C0008D994F849300133DBB2052B84F84930B0
:10186C007FF659AF0023013A84F84930142A0FD877
:10187C00DFE802F00B7E7A76720E6B64605C0E54BD
:10188C0046200E0E0E0E0E191400194B01221A7062
:10189C00184A2978117000232B703CE7164A174B15
:1018AC0012781A70F4E7144B144A1B78C3F1010335
:1018BC001370EDE7002240F6FF6384F84C20A4F887
:1018CC004E30E5E7640700204C070020DC030020C5
:1018DC00D0030020DE060020AC060020ED06002020
:1018EC00D806002004070020970600209806002048
:1018FC00B2060020050700208C05002067000020A0
:10190C0094F84A3001214FF460628B4284F84C10F9
:10191C00A4F84E20BCD184F84830B9E700F05EFB47
:10192C00154B164A1B7801331370B1E7144B012287
:10193C001A70ADE7124B00221A70A9E70E49114B31
:10194C000120002208701A70A2E70B490D4B0020F1
:10195C00012208701A709BE7084B05221A7097E752
:10196C00064B04221A7093E7044B03221A708FE77C
:10197C00024B02221A708BE78C050020B206002065
:10198C008D0500206700002030B52F4DB5F84E3086
:10199C00002B3FD000221846A5F84E201A0A82EAE6
:1019AC0013125340DB4303F00F0343EA0013274A9F
:1019BC00AB6503F00F001913145C515C244844EA26
:1019CC00C134C3F30321C3F30313515CD35C214A29
:1019DC0092F800E044EA812444EA431405EB8E03B8
:1019EC00802200EB8E00EC655A66043013214FF018
:1019FC00010C0CFA01F32340CB4083EAD2120139DB
:101A0C00D2014B1C40F8042FF3D105EB8E050023BB
:101A1C002B6630BD104B1B785BB103460F2240FA8E
:101A2C0002F1012908D0013A082AF8D100226A658E
:101A3C00B4E74FF6FF70F0E7083A40FA02F343EAD6
:101A4C0042206A6583B2A9E7DC03002054610008D8
:101A5C003C040020D30300209706002030B5039CE3
:101A6C0084460AE08C4513DD9C420FD0B1EB6E0F1F
:101A7C000DD0AC450EDC04462A4602EB010EE018F4
:101A8C0094454FEA6E054FEA6000EBDB204630BD13
:101A9C00184630BD691C0346EFE700BF0346401AE9
:101AAC0048BFC81A704700BF034A00235362536AE9
:101ABC008342FCD3704700BF004801400B4A42F6FA
:101ACC00E063002151629362536900EB800043F0A4
:101ADC00010353614000536A8342FCD37823936221
:101AEC00536943F001035361704700BF0048014044
:101AFC00026803FB03F303EB430C22EA0C0201FB29
:101B0C0003F313430360704703FB03F310B404683F
:101B1C0003FB01F103FB02F203EB430324EA03048E
:101B2C000C430460C16810BC21EA03031343C36077
:101B3C00704700BFBFF34F8F0549064BCA6802F4CC
:101B4C00E0621343CB60BFF34F8F00BFFDE700BFD4
:101B5C0000ED00E00400FA0503468A1A0069996852
:101B6C0010B51C6A1A6001FB0201A1421961C4BFC5
:101B7C0021461C6164428C429869C4BF1C61214699
:101B8C00DC68101A04FB00F05C68586104FB02006E
:101B9C005C6A0844A042C3E90620C4BFDC6120464D
:101BAC0064428442C4BFDC612046FFF7F7FB10BDE2
:101BBC0003460069511A1A6A0844904210B518611C
:101BCC00C4BF10461A6152428242C4BF10461A6109
:101BDC005A68196002FB01FC9A69114C8A1AC3E914
:101BEC000521996801FB00F00E4984FB0C4E81FB2A
:101BFC0000414FEAEC7CC017C0EB2130CCEB6E1CE3
:101C0C00D968604401FB0202586ADA61824202DC44
:101C1C004042824201DAD86110BD104610BD00BFAF
:101C2C001F85EB51AD8BDB6870B5C04CC04DB82235
:101C3C002968204682B003F065FA627CA37CE17CC3
:101C4C00207EA2F10102B2FA82F2520984F8B82085
:101C5C00627DA3F10103B3FA83F3A2F101025B09E4
:101C6C00B2FA82F201294FEA521284F8B930E37DBC
:101C7C0008BF84F8BA106A71217DA27D042B28BF9D
:101C8C000223A1F10101A2F10102B1FA81F1B2FA30
:101C9C0082F2EB71A0F1080349095209282B297132
:101CAC00AA7151D8A0F11803182B40F24D81A0F164
:101CBC000C030B2B40F25981A0F10803032B40F2CB
:101CCC00658128899B4BD862637EA3F13202642A1A
:101CDC0044D8994AAB81A2FB03235B0803F10A02A7
:101CEC00EB812A82A37E217F627FE07E287503EB45
:101CFC008303A1F10101A2F10102DB00B1FA81F130
:101D0C00B2FA82F214334909520902206B8284F828
:101D1C00BB1084F8BC2002F04DF86378002B46D140
:101D2C00688A4FF4FA73009340F6B8324FF47A7322
:101D3C004FF49671FFF792FE94F8B130688693B920
:101D4C0084F8C53002B070BD7A4A41F288336B8199
:101D5C00D362637EA3F13202642ABAD99622552348
:101D6C00AA81EB81BEE794F8B33094F8B22094F8D2
:101D7C00B40094F8B710286403EB830302EB8202DF
:101D8C0003EB8303DB0002EB82020120D200AB6386
:101D9C006A4B84F8C5006A6394F8B50094F8B620D1
:101DAC0001FB03F3C5E91102EB6502B070BDA07F26
:101DBC000B2888BF052001F0FDFF94F8202094F833
:101DCC002130E17F94F82300287702F27712520039
:101DDC00EA8294F8222003F26B335B0002F25E522B
:101DEC002B836A8394F8263094F82520A3F1010301
:101DFC00FA32B3FA83F3EA8394F828205B09A1F151
:101E0C000101B1FA81F184F8BF30531F142B4FEA52
:101E1C00511194F8293084F8BD1094F8241098BF0F
:101E2C0085F820205A1E092AA1F1010194F82A20D4
:101E3C0098BF85F82130B1FA81F14909531E84F815
:101E4C00BE10082B4FF0000184F8C0101ED8C2EB56
:101E5C004213C2EB83035B001A3BDBB2C82B85F841
:101E6C00222000F29F8085F823309AB2A98C314E43
:101E7C00607E1144A984E98C1144E984716C0B4394
:101E8C007364131802EB5002AB81EA8194F82B3087
:101E9C00A3F14602462A98BF85F8283094F82C30D6
:101EAC005A1E622A04D85B0001226B8584F8C1207B
:101EBC0094F82D305A1E092A98BF85F82C3094F8C6
:101ECC002E30092B06D8042B0CD8DFE803F0037D49
:101EDC00790B70001A4A0023012184F8C23084F86F
:101EEC00C330117094F82F30688A164A297DA3F1FB
:101EFC000103B3FA83F35B09B0F5967F84F8C43021
:101F0C003CBF002385F82D302023B3FBF1F1A2FB5D
:101F1C000032094B5209B2FBF1F2EA85A3FB002314
:101F2C00DB08B3FBF1F32B86FBE600BFD4040020E7
:101F3C0000000020002C0140ABAAAAAAA086010038
:101F4C00240400201F85EB5140F6C413009330226B
:101F5C0041F288331821FFF781FD0346207E2B8147
:101F6C00A0F10C030B2B3FF6A7AE41F28833009384
:101F7C00182242F210730C21FFF770FD0346207EED
:101F8C002B81A0F10803032B3FF69BAE41F64C537B
:101F9C000093102243F698230721FFF75FFD80B2D0
:101FAC0028818FE6C822134685F823205EE709496D
:101FBC00094A01230B700021117084F8C23091E79B
:101FCC00012384F8C3308DE7034A012384F8C2301F
:101FDC00137087E7260400202404002000B5214854
:101FEC00214B90F8B8C090F8B92090F8BA1093F83B
:101FFC0064E080F801E0ACF1010CA2F10102A1F166
:10200C000101BCFA8CFCB2FA82F2B1FA81F14FEA0E
:10201C005C1C5209490980F811C08274C1741A7988
:10202C0093F805C0997993F807E080F817E0A2F1CE
:10203C000102ACF1010CA1F10101B2FA82F2BCFA7D
:10204C008CFCB1FA81F1520949094FEA5C1C02750A
:10205C00817580F815C01A685DF804EBB82102F0A0
:10206C00F5BF00BFD40400200000002000B5124AC8
:10207C0092F8CC10B2F89831D2F8C80002EB410CAF
:10208C000131C9B26329BCF8D0E0ACF8D0301844A7
:10209C0084BF002382F8CC30084B98BF82F8CC1058
:1020AC00A0EB0E00C2F8C800A3FB0030C0F34F1029
:1020BC00A2F89A015DF804FBD40400201F85EB51B3
:1020CC0008B502F097FF0E4B93F865203AB140B972
:1020DC000C4A92F89C31013382F89C3108BD0028DF
:1020EC00F6D1084A93F8661092F89D310133DBB2B1
:1020FC00994282F89D31F1D2002382F89C3108BDBF
:10210C0000000020D404002038B5284C94F8673027
:10211C00012B3BD094F86830254D5A1E12F0FF026B
:10212C0022D084F8682003F0010384F8653072B67D
:10213C0095F89F312BB362B602F078FFD5F8A02149
:10214C00E16E40F2A4639A4284BF012384F86930A3
:10215C0094F8683005EB4303002285F89C2185F840
:10216C00A421A3F8A61138BD0123062284F8682007
:10217C0085F89E3184F8653072B695F89F31002B46
:10218C00D9D194F8680003F07FFBD4E794F8682069
:10219C00074D0132D2B2062A99BF84F8682002F0AA
:1021AC00010384F8683085F89E31BEE700000020FA
:1021BC00D40400201B4AD36823F0010310B5D3606C
:1021CC00FFF7A2FF1849194CCB6EB4F8B40194F880
:1021DC00C42003EB430303449808C866C2B991F8C2
:1021EC007020580912FB00F292B291F86910A4F811
:1021FC00B821C2EBD303A4F8BA3181B1D4F8BC3105
:10220C0042F20F7293429CBF0133C4F8BC3110BD33
:10221C0094F8B62100FB02F2C2F38F12E5E702F04C
:10222C00FDFEEBE70044014000000020D404002038
:10223C0070B5254ED6F8A0317D2B15D9234B5B6A92
:10224C007C2B09D8B6F8C031B3F5167F04D2D6F87A
:10225C00BC31B3F5FA7F19D396F8C2310133DBB236
:10226C00642B86F8C23128D8194D95F871300024AA
:10227C0023B90CE095F87130A34208DD02F0BAFEE8
:10228C0095F86530834204F10104F3D170BD72B648
:10229C0002F0B8FE0D48B6F8BA11426A0D4BA6F81A
:1022AC00B4210131002242625A62D9621A61DA68A1
:1022BC0042F00102DA6062B670BD02F0A3FE0023A8
:1022CC00C6F8BC3170BD00BFD40400200010004023
:1022DC00000000200044014070B5CE4C94F8B93099
:1022EC0082B0002B00F0C88094F8C230002B00F0B4
:1022FC001A81C94DB4F8C421B2F5836F80F0D08136
:10230C00A2F130039BB2B3F57A7F11D294F8B810D6
:10231C0095F86760C1F10100864200F08C8395F856
:10232C0072105B009BB2C1F12F010B44A4F8C631B3
:10233C002F2A00F2A680002394F8CB21A4F8C631F2
:10234C0084F8CA3195F873309A4200F2A18094F85F
:10235C00BA60002E00F0BF80B4F8C6011D2800F250
:10236C0085810023A4F8CC3195F8203003EB83034E
:10237C00B0EB830F4FEA830180F2848194F8C9316A
:10238C00002B40F0448194F8BA102E22502313FBFA
:10239C000123B4F8CC21934280F28D8094F8D8318B
:1023AC00002B00F02F8194F8C331002B00F05C83DC
:1023BC0094F8BA30002B00F0A382EB89B4F8CC016E
:1023CC004FF4FA620092283340F2FF728921FFF732
:1023DC0045FBA4F8DC0194F8BF3094F8BA10002B3C
:1023EC0040F00781B4F8CC6184F89F3150222E2341
:1023FC0012FB0133B3425EDA2E2E40F2158294F8B2
:10240C00BC201E23D340D4F8BC21934240F20C8252
:10241C00B4F8DC31AA8993423CBFA4F8DC21134602
:10242C00EA8C9A423CBFA4F8DC211346B5F876201E
:10243C009A4294F8C13038BFA4F8DC213BB1B5F90D
:10244C007830B4F8DC219A42C8BFA4F8DC31D4F857
:10245C00E85100212846FFF761F8002800F0D780EA
:10246C002F2E40F2D4802846FFF788F8B4F8DC31E0
:10247C001844A4F8DC01CAE0B4F8C431664DA4F8E1
:10248C00C63194F8CB2195F873309A427FF65FAF42
:10249C00AB79002B3FF45BAF03F0B8F902F0B2FD5F
:1024AC0000226623A4F8CC2184F8CB3194F8C931EE
:1024BC00002B40F0AC8094F8DE31002B00F0B7809C
:1024CC00013B042B00F2B080DFE813F0AC003B02C0
:1024DC0038023502AC0094F8CE31002B00F0DB80D2
:1024EC0094F8C530002B40F05981D4F8D4614B4995
:1024FC003046FFF713F8002840F0F2813046FFF722
:10250C003DF8A4F8CC0146493046FEF7E9FF002817
:10251C003FF434AF94F8C9313022A4F8CC21002B0D
:10252C003FF43CAF73E094F8BF203B4DB4F8C401CA
:10253C00002A00F0EF802E7F760006F57A71884233
:10254C001DDD94F8B86095F86720B24200F01B824C
:10255C0094F89F31002B40F01B81002384F8C83184
:10256C0040F2FF7300934FF4FA622F23FFF776FAD1
:10257C002E7F0346B4F8C401A4F8C6317600C6F524
:10258C007A72824222DD94F8B83095F86760C3F114
:10259C0001018E4200F0258294F89F31002B40F00F
:1025AC00F7802F230021009340F2FF7384F8C811A9
:1025BC00FFF754FA2E7F03467600B4F8C401A4F852
:1025CC00C631C6F57A739842C0F2E28006F57A7687
:1025DC00B04200F3DD8094F89F210023A4F8C631AB
:1025EC00002A00F0D580012284F89F3184F8C8219C
:1025FC00CEE02E22502313FB0123B4F8CC219342BE
:10260C00BFF659AF94F89F61002E00F0088102B01C
:10261C0070BD00BFD40400200000002000E0FF4487
:10262C000000404201F004FD002384F8DE312B79D8
:10263C00002B4BD194F8C321A4F8DC31002A40F0D4
:10264C00F88094F8BB30C4F8BC21012185F86910DE
:10265C00002B40F0EC8094F89F31002B00F0378277
:10266C0094F8BF30002B40F0ED80D0E71E283FF4EB
:10267C007BAE95F8202002EB82029200904211462C
:10268C00C0F2C18040F2FF720092A023FFF7E6F97E
:10269C00A4F8CC0172E6B4F8C631A4F8CC316DE6DE
:1026AC0094F8B83095F86710994200F0AB8195F822
:1026BC007200A2F58361490089B2C0F12F00A2F12A
:1026CC00300301449BB2A4F8C6111CE694F8C33144
:1026DC00002B40F0CE8094F8BB20C4F8BC3101260E
:1026EC0085F8696084F89D31002A00F0C08094F868
:1026FC00BA00002840F0BF8095F8213003F2DE3399
:10270C005B00A4F8E03102F0E3FF94F8BA0084F81F
:10271C009F61B2E02A7F520002F57A71884240F341
:10272C00E48094F8B83095F867209A4200F00C8158
:10273C0040F2FF7300934FF4FA622F23FFF78EF9E8
:10274C002B7F02465B00B4F8C401A4F8C621C3F584
:10275C007A72824240F3E98094F8B83095F8676059
:10276C00C3F101018E4200F020812F230093002140
:10277C0040F2FF73FFF772F92B7F02465B00B4F84F
:10278C00C401A4F8C621C3F57A72904280F2CD80C0
:10279C0094F8C230002B3FF474AEABE5D5E90D32A2
:1027AC002F210092B4F8C60140F2FF72FFF756F9E0
:1027BC00B4F8C6112A7DCC4BA4F8D0012E2980B2D6
:1027CC004FEA5202B3FBF0F0B0FBF2F0A4F8D201E6
:1027DC0040F2A480D4F8D461C4493046FEF79EFE82
:1027EC00002840F05B813046FEF7C8FEA4F8CC010F
:1027FC00BF493046FEF774FE00283FF4BFAD3023CE
:10280C00A4F8CC31BAE5A02300931E212F23FFF7A7
:10281C0025F90346A4F8CC31B4F8C601A4E5B4F804
:10282C00CC612E2E3FF6EBADB4F8DC31FEE503F0B7
:10283C004DF994F8BF30002B3FF4E4AE94F89F317F
:10284C00002BECD0B4F8C4114FF47A70FFF726F9D2
:10285C002A8900F57A739BB2013A9342A4F8E031CD
:10286C00C0F23E8103F032F994F89F61CCE602F09D
:10287C00CDFF94F8BA0094F89F6195F86830013B4D
:10288C00C3EB0312B5F8743003EB82031AB2B2F542
:10289C00B47F9BB2A6BFA3F5B4739BB2A4F8E2219C
:1028AC0003F1770212B2A8BFA4F8E231B2F5B47FFB
:1028BC00A8BFA3F1F102A4F8E42103F1EF0212B2D4
:1028CC00B2F5B47FA6BF793BA4F8E631A4F8E621B3
:1028DC000023012808BF84F8C901A4F8DC3193E671
:1028EC0040F2FF73A4F8CC310DE6C2F57A72904237
:1028FC00FFF632AF0023A4F8C63184F8CA3147E79B
:10290C004FF4FA62EB89B4F8CC0100922F2140F21B
:10291C00FF72FFF7A3F8A4F8DC015CE50023A4F830
:10292C00CC61EE63C4F8D431C0E503F57A7383420D
:10293C00FFF62EAFDEE701F00DFB75E601F0D8FBDC
:10294C0072E601F0A5FB6FE6688EEA6E904280F0AD
:10295C00AA80B4F8C021C72A00F2A580C3F10103F4
:10296C000026012285F86730C4F8BC6185F869201F
:10297C0002F048FB297FB4F8C40184F8CA6149000D
:10298C0001F57A71D4E694F8C861A4F8C6314FF019
:10299C00010C84F89FC1002E3FF4FAAEACEB02029E
:1029AC0084F89F3185F86720D7E5688EE96E8842F8
:1029BC0080F08380B4F8C011C7297ED8012200268C
:1029CC0085F86920C4F8BC6185F8673002F01AFB01
:1029DC002A7FB4F8C40184F8CA615200C2F57A7235
:1029EC00C3E694F8C86100214FF0010CA4F8C6119D
:1029FC0084F89FC1002E3FF4CBAE85F8673084F885
:102A0C009F11CEE5698EEA6E914240D2B4F8C02196
:102A1C00C72A3CD80122C3F10103002685F869209E
:102A2C0085F86730C4F8BC6102F0ECFAB4F8C42144
:102A3C0084F8CA613BE66A8EEB6E9A4220D2B4F8F7
:102A4C00C031C72B1CD80123002685F86930C4F887
:102A5C00BC6185F8671002F0D5FAB4F8C42184F88B
:102A6C00CA61A2F130035AE402F0D0FE95F8693045
:102A7C0083B3AB89A4F8DA31012284F8C32197E43B
:102A8C0094F8C931002BDED1A4F8C43153E494F886
:102A9C00C921002ABED1A4F8C4214CE440F2FF7332
:102AAC00A4F8CC31A4E694F8C921002A7FF456AFDF
:102ABC004FF47A70A4F8C4013AE694F8C9110029CD
:102ACC007FF47CAF4FF47A70A4F8C4014DE602F0A9
:102ADC009DFEAEE694F8C33163B102F09FFAC8E7ED
:102AEC0002F0F6FD8EE500BF0087930300E0FF4483
:102AFC0000004042FFF708FB054B42F2107141F217
:102B0C008832E9665A62012384F8C331E5E700BFD5
:102B1C000010004010B50E4C94F8EC31012B0DD088
:102B2C00022B03D0BDE81040FFF7D6BBB4F8F00180
:102B3C00FEF72AFF002384F8EC3110BDFEF778FD78
:102B4C00002384F8EC31BDE81040FFF7C5BB00BF93
:102B5C00D4040020F8B54F4E4F4F96F8671000295B
:102B6C0077D1B7F8E23101331AB2B7F8E431013357
:102B7C00B2F5B47F1BB2B2BFA7F8E221A7F8E211FD
:102B8C000A46B3F5B47FA8BF0023A7F8E431B7F821
:102B9C00E63101331BB2B3F5B47F77DAA7F8E6312F
:102BAC0006EB4202B6F84C13B2F97C3030893B4D3F
:102BBC003B4C0B4400FB03F385FB0312D81796F830
:102BCC002C30C0EBE21003FB00F0C31784FB002099
:102BDC00C3EBA00080B202F0DDFCB7F9E431B6F82B
:102BEC004C0306EB4303B3F97C2096F82C300244DB
:102BFC00308900FB02F285FB0201D017C0EBE1101B
:102C0C0003FB00F084FB0023C017C0EBA30080B2D1
:102C1C0002F0C6FCB7F9E621B6F84C0306EB42020B
:102C2C00B2F97C3096F82C200344308900FB03F376
:102C3C0085FB0315D817C0EBE51002FB00F084FBF5
:102C4C000034C017C0EBA40080B2BDE8F84002F01D
:102C5C00ADBCB7F8E221B7F8E431013A12B2013B4E
:102C6C001BB2002AB8BF40F26712002BB8BF40F26B
:102C7C006713A7F8E431B7F8E631A7F8E221013B76
:102C8C001BB2002BB8BF40F2671387E70023A7F8ED
:102C9C00E63185E700000020D4040020D34D6210FB
:102CAC006766666638B5234D2349EA6E4B6A234C3A
:102CBC0002EB420212FA83F2A4F8B43100234B6205
:102CCC0053095B009BB2A4F8B831C3EBD2039BB29F
:102CDC009208D4F8BC01EA66A4F8BA3101E00428E1
:102CEC0002D94A6A9A42FAD3FFF70EFAD4F8BC31E9
:102CFC0094F8BC0094F8BF100022013384F89C2196
:102D0C0084F89D2150EA0102C4F8BC3105D1EA6E69
:102D1C0040F213539A4206D938BD132BFCD9EB6EF3
:102D2C00B3F5FA6FF8D8002385F86930BDE8384060
:102D3C0002F074B90000002000100040D404002000
:102D4C00F8B5BE4CB4F8F611B4F8F401B4F8F821A7
:102D5C0094F8D831B4F8DC51A4F8C0510131A4F87E
:102D6C00F61194F8FA11013001320B43A4F8F40176
:102D7C00A4F8F8213ED194F8FB21002A3AD0B4F8FB
:102D8C00C651002D40F0A181B4F8FC3101339BB247
:102D9C0044F620618B42A4F8FC312BD9B4F8FE31F7
:102DAC001E2B40F2C78194F8BE30012184F8D81153
:102DBC00002B00F0C481B4F80012A1484B08A0FB12
:102DCC000323DB09B1F5B97F84F8FA310DD39D4F9C
:102DDC004AF6AA2601F0F6F86420FEF76FFE94F886
:102DEC00FA313E600135AB42F4DC94F8C3300BB9D8
:102DFC0084F8BF3094F8BD3073B1934AB4F8023202
:102E0C0092F84E2301339BB202EB8202B3EB820F9A
:102E1C00A4F8023200F3B78094F8C931002B38D1F2
:102E2C00894D95F8693023B194F8C331002B40F0EB
:102E3C003281B4F8F831142B31D895F8A833002B23
:102E4C0040F0A880B4F8C01194F8D83123B194F8AC
:102E5C00C331002B40F00E8194F89F316889002B10
:102E6C0000F0BF802B89B4F8E0215D1C774B00FB90
:102E7C0002F283FB023CD317A3EBEC132B449BB263
:102E8C00A4F80832724AA4F8DA11C2E90D33D06200
:102E9C00D363B4F80A320133A4F80A32F8BD94F8BB
:102EAC00C1300022A4F8F82123B194F8C331002BCF
:102EBC0040F0198194F8BC30002B40F09C8094F8C1
:102ECC00CE31002BB9D094F8C331002BB5D0B4F867
:102EDC0000226B8A5F48B4F8D0615F4F02FB03F3AA
:102EEC00A0FB03235B09C6EBC620B0FBF3F0FEF797
:102EFC0055FA2B7DD4F8F0115B0801FB03F3324635
:102F0C00564991FBF3F106465548FEF751FEFEF784
:102F1C0045FA3146FEF78EF939460646FEF7FEFABB
:102F2C0038B9504F30463946FEF7DAFA002800F02F
:102F3C000C81C4F8D471D4F8BC31632B3FF67DAF4F
:102F4C0095F8A8330022EA64002B3FF47BAFB4F869
:102F5C00DA3101210A4685F8A9138C46B4F8C01160
:102F6C00C81A90422EDC581A904240F3B580A3EB5D
:102F7C000C0399B2EA79A4F8C011002385F8AA339E
:102F8C0085F8702060E70122002384F80422A4F85D
:102F9C00023241E7D4F8BC31952BB4F8DA31D8D9E8
:102FAC00952BD6D9D4F8A021B2F5FA7F8CBF042189
:102FBC0010210A4685F8A9138C46B4F8C011C81A1A
:102FCC009042D0DDEA6E634499B2B2F5FA7FA4F870
:102FDC00C0117DD9EB7985F87030012285F8AA23D0
:102FEC0032E71A4A00FB01F3A2FB0323C3F3CF130E
:102FFC00A4F8083246E794F8C331002B3FF41DAF18
:10300C00B5F87C23E96E1848184FFEF7A5FD184952
:10301C00FEF756F8D4F8E811FEF70CF939460646D7
:10302C00FEF77CFA38B9002739463046FEF762FACB
:10303C00002800F08780C4F8E87140E7D404002031
:10304C00B9D31FB10030004000000020D34D6210F6
:10305C00002C01401F85EB5100E0FF4400879303D7
:10306C003C0000200000404280030020000016437A
:10307C0017B7D138B4F8CC312F2B7FF6EDAE688969
:10308C00334A00FB01F3A2FB0323DB0901339BB2A0
:10309C00A4F80832F6E601F0B5FFFFF711F894F842
:1030AC00A431002B7FF4C5AE95F8653094F89C21C3
:1030BC00002B39D095F84F339A427FF6BAAE0123E4
:1030CC0084F8A431FFF7EEFDB3E6A4F8FC3191E6E9
:1030DC00002385F8AA33B7E6EA7985F87020002337
:1030EC0085F8AA33B0E66B8DB4F906121948642240
:1030FC0003FB02F2FEF730FD1749FDF7E1FFFEF787
:10310C0017FAB5F87830E9891B1A1BB21A468B42AC
:10311C00A5F878306B89BCBF0AB2A5F87820934229
:10312C00B8BFA5F87830C5E695F850339A427FF6CB
:10313C0080AEC4E784F8FB51A4F8FC515AE600F0C9
:10314C0041FF52E6C4F8E861B9E6C4F8D461F2E68E
:10315C00D34D62105403002017B7D1382DE9F04F2E
:10316C0085B002F071F84FF47063CB4AD3F8E010DD
:10317C00914205D1C94AD3F8E410914200F077830B
:10318C00C74DC84C02F0A4F902F026FAFEF74CFD2C
:10319C00E378022B02D12379102B0CD00222C24BE4
:1031AC00E2701022227107CBC04EC4F8050071608A
:1031BC00B260FEF713FF94F8B8302A792989698137
:1031CC00013B18BF012385F867300AB984F8BA208F
:1031DC0094F8BF30B3B1E889298AAA890023012663
:1031EC004FF47A77323032313232AF84E88129822F
:1031FC0084F8B96085F82D6084F8BA306B712B7146
:10320C00AB71AA8100F064FE0023A4F8FE3102F039
:10321C0081F8A74B4AF6AA221A6001F081FF94F8B4
:10322C00C53013B1012384F8CE3102F005F8A04F5C
:10323C00DFF880B2DFF88092DFF880824AF6AA26A7
:10324C00B4F8AA11B4F8A831B4F8AC21B4F8AE01B2
:10325C000B441344B4F8B011B4F8B2213E600344EB
:10326C000B44134404336A795B10C4F8F031002A20
:10327C0040F0A781B4F80A3242F21072934209D995
:10328C0094F8D811002940F0D98249F64042934273
:10329C0000F2F982B4F8F42144F620639A421BD967
:1032AC00B4F906A25046FEF779F85946FDF708FF27
:1032BC00D4F80C12FDF7BEFF99F80030C4F80C02DC
:1032CC00022B00F07282032B00F06082012B00F0C5
:1032DC0053820023A4F8F431D4F8BC21B2F57A7FE0
:1032EC0040F229810021B4F8C63184F8CB11C72BE8
:1032FC0040F2E38194F8BA1011B19F2B40F228816F
:10330C0094F81112002900F0C080B3F5C87FC0F00A
:10331C002681D4F8F03194F89E0188FB03C1A1EB0F
:10332C00E371C4F8A01110B10A2A00F2F58194F8E7
:10333C001932002B00F08580EB6E322B40F281802D
:10334C005F4B1022002183F80B1383F8152383F8AD
:10335C000C2394F80432002B40F0818094F81C323A
:10336C000133DBB2C82B84F81C3200F2478194F88D
:10337C00C9314FF0000A84F8C2A1002B40F0A8809C
:10338C0094F8C3314F4AD4F8F0114F4892FBF1F244
:10339C0013FB02F39BB2A0FB032095F82D20A4F89D
:1033AC001A32C008A4F82A02002A40F0978194F837
:1033BC00100295F828104FF4FA638842A5F876307D
:1033CC0000F29D81D4F8BC31632B00F20481EB6ECA
:1033DC00B3F5FA7F40F2FF800C2385F87130172388
:1033EC0000934FF4FA620D23B4F8C0016421FEF788
:1033FC0035FB364A526A84F8B6014AF6C8739A42CB
:10340C007FF61EAF94F8C3A1BAF1010F7FF418AF89
:10341C0094F8CB31013384F8CB3101F0F3FDB4F8DF
:10342C00CC3185F869A02F2B05D8002384F8C33143
:10343C0041F28833EB660023C4F8BC31FFF732FC51
:10344C00FEE61F4B0022102183F80B1383F8152383
:10345C0083F80C2394F80432002B3FF47FAFD4F89C
:10346C000C02FEF78BF8B4F81A12B4F8062200918D
:10347C0083B2B4F8001294F8100202F07DFB02F053
:10348C006DFB002384F8043268E7952B94BF64230A
:10349C000A2385F873303CE7DAE32559D963B84E33
:1034AC0000000020D404002094610008D9040020FE
:1034BC0000300040610B363B280400205655555512
:1034CC0000E100E0C0270900CDCCCCCC00100040BE
:1034DC00B4F8CC31302B4AD994F8D821002A46D0F4
:1034EC00313B572B00F26F8194F82C32002B40F0BB
:1034FC00FB81FFF72FFB95F814E0B4F8CC01782290
:10350C00302141F6583340F22A3CB3FBFEF3BCFBAE
:10351C00FEFCCDF800C0FEF7A1FAA5F8B00380B20E
:10352C00FEF7C2FAB5F8B0234FF41673B3FBF2F3FF
:10353C00A4F81A3284E6B4F8C631A3B9642A84F824
:10354C00CB3100F2BA8094F8BA1000293FF4D8AE0F
:10355C00002184F8CB1194F81112002995D0002386
:10356C0084F8CB31D5E6642A7FF6C4AEBFE694F876
:10357C00BB304FF0010A84F82CA2002B00F0A7807E
:10358C002B8995F82110A3F1130202EB41026989F2
:10359C0092B2A4F8C02101FB02F2B2FBF3F2534445
:1035AC009B1AA4F8083202F093F8B4F80822C34B23
:1035BC0084F89FA1C3E90D22DA630023A4F81A3220
:1035CC003EE62B890093E86E5B08C8226021FEF76B
:1035DC0045FA68814EE60C230093D4F8A00103232E
:1035EC004FF4FA726421FEF739FAEB6E85F871002C
:1035FC00312B9CBF022385F87130F0E601F050FBB3
:10360C000121AF4800F0FAFEB4F81E0201F0E8FB0D
:10361C00B4F82222AB4BA4F8200240F6E44A0AFB91
:10362C0002F2A3FB0213D21A03EB5203B5F8AC233C
:10363C00A54984F81002DB0A02FB03F3B4F800225C
:10364C00A1FB0313C2EBC20202EB5313DB10A4F871
:10365C000032FEF70BFD9D4BC4F824020AFB00FA66
:10366C00A3FB0A3A4AF30F2ABAF1000FBCBF00239E
:10367C00A4F8063294F8BE30A8BFA4F806A21BB377
:10368C0094F8FA31E98BB4F8002201FB03F39A4267
:10369C0017DAB4F8282294F8C9318D48013244F66F
:1036AC00206192B200FB03118A42A4F8282200F395
:1036BC002C81002284F81C225BE6002184F8CB11BB
:1036CC0018E60023A4F8283294F8C931F1E77B4AB4
:1036DC00C2E90D33D36302F099F86EE7B5F8AE3357
:1036EC000093E98DAB8C2A8EFEF7B8F995F828106B
:1036FC00A5F8760094F8100288427FF663AEB5F810
:10370C00AE33012200925B0801F10A020A39FEF77E
:10371C00A5F9A5F8760055E6D4F81402FEF7BEF923
:10372C00D4F8A031B0EB530F1BD9B3F5FA6F18D204
:10373C0094F81822013284F8182294F8B920002148
:10374C00C4F8BC119AB9B4F8CC212F2A0FD9002295
:10375C0084F8C321AA895208A4F8DA21012285F839
:10376C006920002284F89E21C4F81432DFE5EA6E49
:10377C00B2F57A7FEED9EAE794F81032554A43F461
:10378C0000731380022389F80030A2E5B4F80032EC
:10379C004D49504AA1FB0313C3F3C70343F48063A1
:1037AC001380012389F8003093E5474A5FFA8AF3C6
:1037BC00A2FB03231B09474A43F4C0631380032372
:1037CC0089F8003085E5012384F82C32FFF7C2F923
:1037DC00B4F8CC31C82B04D95023A4F8E2A1A5F835
:1037EC00B033B5F8B003FEF75FF9B4F9E231002B52
:1037FC007FF426AD384984F8C931012284F89F3111
:10380C0042F22833EB66C4F8A031C4F8143285F8C0
:10381C0069204B6294F8BC3084F8C32195F8B2232C
:10382C0085F868201422C4F8BC2113B12B8AA4F8A3
:10383C00DA31FEF769FC01F0BFFE01E501F0E6FFAD
:10384C001E4B0025C3E90D55DD6384F8D851A4F84F
:10385C00CC5184F8FB51A4F8FE5101F0B5FE1F4881
:10386C004FF48072294602F05BFCFEF763F993F883
:10387C00EC301B4D2B2B5CD0352B57D01F2B04BFA2
:10388C00184B2B607DE4039101F0C0FF03990B4BA7
:10389C0084F8D811C3E90D11D963A4F8CC1184F8BC
:1038AC00FB11A4F8FE11039101F08EFE03990B4855
:1038BC004FF4807202F034FCD7E700BF002C0140BB
:1038CC0000240140010110001F85EB51FF04EC4F57
:1038DC007CFCFFFF2A04002000100040640700203D
:1038EC0000000020007C0008134AD36823F0010379
:1038FC00D36001F087FB114BC3E90DAAC3F83CA0C0
:10390C0002F022F984F82CA2F3E54FF0000AA4F897
:10391C00CCA101F07BFF01F075FB94F8C93184F860
:10392C00C3A1A4F8FEA184F8D8A1C2E6044B2B6075
:10393C0027E4044B2B6024E400440140002C01409C
:10394C0000F8000800F80108F0B5604CD4E900025A
:10395C00101A6FF4487240F2765382189A4283B070
:10396C002AD85B4E5B4D002333802B78002B3CD048
:10397C006B780146ABB9AB78002B00F08E80A88831
:10398C00554F01333988AB70FEF788F8322866D969
:10399C0000223B882A706A78AB804AB1D4E90031A6
:1039AC00C91A40F2E14399424DD9AB794B2B77D8E8
:1039BC000023A868338004E04649484B88680022FD
:1039CC001A804749474A0B881268A0EB030C9445B0
:1039DC0003DD13440B8003B0F0BD1C1AA242BABF26
:1039EC009B1A0B80088003B0F0BD3F4A147874B169
:1039FC003E4A128890421AD83D494FF47A7409888D
:103A0C000094FEF72BF8A86000233380D9E7324BE3
:103A1C001A88374B198840F2FF7300932F23FEF757
:103A2C001DF83028CEBFA860AC602046ECE72A4BCE
:103A3C00511C1A884FF4FA63009340F2E933FEF7F5
:103A4C000DF8A860E0E72A48AB790288C2EBC20205
:103A5C0001331144DBB2C908AB710180A6E73B8886
:103A6C006268C3EBC3012368D31AAA780B44C3F36F
:103A7C00CF03322A3B808ED9193B9BB23B80A3F2F9
:103A8C00D6631C4A03EBD3735B1082F821300123FD
:103A9C006B7000F0CDFA3B887DE780B2A8806FE7B1
:103AAC00134A1449138819339BB21380A3F2EE23E3
:103ABC0003EBD3735B10002481F820302C70FEF7DD
:103ACC008DFAAC7100F0E4FA72E700BF64070020D5
:103ADC00DE0600203407002018000020D20600204B
:103AEC0098060020C80300208D0500201A00002035
:103AFC0016000020D40400201A4A9388591E02296B
:103B0C0030B413D8184BD9683B290DD80121174D67
:103B1C001748197400232B70164C174B21700E2567
:103B2C00057020209071197030BC7047043B042B39
:103B3C00FAD80D4BD9686329F6D80D480D4D0B4CAE
:103B4C004FF0030C83F810C00B4B4FF0070C012106
:103B5C0080F800C02020297021709071197030BC41
:103B6C00704700BFC803002034070020D203002098
:103B7C00D303002096050020CF060020F8B5284B73
:103B8C00284F1968002544F6206E1A46A7F804E061
:103B9C0003F17804AC462E4652F8043F8B42A3EB5B
:103BAC000100194606D070453CBF1FFA80FE012665
:103BBC0084440125A242EFD10EB1A7F804E00DB167
:103BCC004FEA5C15184C194A2378D560012B23D089
:103BDC00174D2B78012B15D02278134311D1FFF7F9
:103BEC008BFFBB88C93B44F656529BB2934208D814
:103BFC0001231049104A2B70772008700221B971EB
:103C0C001370F8BDBA88C93A44F6565192B28A423A
:103C1C00F7D80849084AEFE7FFF76EFFD8E700BF6F
:103C2C0064070020C80300209605002034070020FC
:103C3C0097050020D2030020CF06002070B5504C11
:103C4C00237813B14F4B1B7833B94F4B1B78002B98
:103C5C004FD0012B0AD070BD4C4B1B78002B35D0AC
:103C6C0001F05EFA4A4B02221A7070BD454B1B786C
:103C7C00002B31D1474D2B78012B6FD0464B1B7845
:103C8C00012B62D02378002BE5D12B78002B3AD076
:103C9C004249434B4A7C072A36D81888052833D921
:103CAC00404C4D69E06F24680132D2B22844001BAD
:103CBC00082A4A74486127D1C0F3CF023A4CC0F3AA
:103CCC00CF101518101A258108831DE001F062FA37
:103CDC002F4B01221A7070BD2C4B1B787BB1334BD0
:103CEC001888FDF751FEFDF7A3FCBDE8704001F00C
:103CFC0017BAFFF743FFBDE8704001F011BABDE8F9
:103D0C00704001F047BA264B294C208830B9234A21
:103D1C00127842BB1A8801321A8070BD40F2DC5214
:103D2C00002690421E8096D91C4D698BFDF7B6FE7D
:103D3C0032281ED82B7F0133DBB2322B2B7701D9E3
:103D4C006E7896B123886B8370BD01F06DFA164BBB
:103D5C0088B103229A7101F0E3F993E7FDF768FC4F
:103D6C0001F0DEF98AE7188070BD00F0C1F901237B
:103D7C002B702E77E6E702229A71FFF7E5FDEAE752
:103D8C00AC060020ED060020CF06002060070020C6
:103D9C00C00600209605002097050020340700205F
:103DAC00D206002064070020C8030020C4060020AF
:103DBC009A0600200B28034B28BF0B2040001870DC
:103DCC00704700BF510700202DE9F84F354C364E97
:103DDC00DFF8D880032001F057FD04F17C070023A5
:103DEC0018E094F835503249DFF8C8B0C3EBC31073
:103DFC00F7224FF47A6A0CEB400080B212FB05A25A
:103E0C004DBBC1E90D55CD63FDF758FE2B46023471
:103E1C00BC4211D04AF6AA22C8F8002094F834C04B
:103E2C004FF00009BCF1FF0FA6F80090D9D1023475
:103E3C000133BC42DBB2EDD101F0E8FC1E481C4A58
:103E4C0000881A4900239362D0624AF6AA22338072
:103E5C000A60BDE8F88FBBFBF2FA4FF00A0E174A66
:103E6C00174DB2FBFAF290B2C1F828E0C8622A787A
:103E7C0000FB02F2FE2010FB03C0124BA3FB02322C
:103E8C00114BB3FBFAFA114B0AFB00F0120BA3FB1C
:103E9C000030C1E90D22CA63C0F34F10FDF70EFECE
:103EAC004B46B4E7D4040020DE060020003000406E
:103EBC00002C01408096980008000020001BB700E1
:103ECC00510700205917B7D1A08601001F85EB516F
:103EDC0010B572B61A4B1B6893F83030FF2B07D015
:103EEC00FFF772FF174A184B1288DA6262B610BDE0
:103EFC00154C164B41F28832E2621B78E363C4E93D
:103F0C000D33032001F0C0FC3723A362C820FDF75A
:103F1C00D5FD052001F0B8FC2823A362C820FDF7CD
:103F2C00CDFD062001F0B0FC1923A362C820FDF7DB
:103F3C00C5FD01F06BFC064A0023A3621380D1E798
:103F4C000000002008000020002C01405107002038
:103F5C00DE06002070B5164C41F28833E36272B66F
:103F6C00144D154B3C224AF6AA262E60A2621B78F1
:103F7C00E363C4E90D33012001F086FC4B20FDF70F
:103F8C009DFD5023A3624B20FDF798FD5A23A3629D
:103F9C004B202E60FDF792FD01F038FC074A0849D2
:103FAC0012880023A3620B80E26262B670BD00BF70
:103FBC00002C014000300040510700200800002078
:103FCC00DE06002010B572B6144C154A154B4AF695
:103FDC00AA2141F28830E06211605022A2621B7863
:103FEC00E363C4E90D33032001F04EFC6420FDF7BC
:103FFC0065FD4623A3626420FDF760FD2823A362C0
:10400C006420FDF75BFD01F001FC074A07491288AB
:10401C000023A3620B80E26262B610BD002C01404B
:10402C00003000405107002008000020DE06002070
:10403C0010B5124C124B41F288313222E162A2626D
:10404C001B78E363C4E90D33022001F01DFC9620BC
:10405C00FDF734FD0B4A4AF6AA211E231160962067
:10406C00A362FDF72BFD01F0D1FB074A074912882B
:10407C000023A3620B80E26210BD00BF002C014044
:10408C00510700200030004008000020DE06002010
:10409C0010B5124C124B41F288312822E162A26217
:1040AC001B78E363C4E90D33022001F0EDFB96208D
:1040BC00FDF704FD0B4A4AF6AA2150231160962005
:1040CC00A362FDF7FBFC01F0A1FB074A074912882C
:1040DC000023A3620B80E26210BD00BF002C0140E4
:1040EC00510700200030004008000020DE060020B0
:1040FC002DE9F041154D41F28833EB6272B6144B49
:10410C00DFF850801B78144FEB63C5E90D3377242F
:10411C004AF6AA26A7FB04300009C8F8006001F093
:10412C00B3FB63100A33AB620A20023CFDF7C6FCFA
:10413C00631CEFD101F06AFB084A0949128800237D
:10414C00AB620B80EA6262B6BDE8F081002C0140E4
:10415C005107002000300040CDCCCCCC0800002012
:10416C00DE060020002103E00B4B5B58435004316A
:10417C000A480B4B42189A42F6D30A4A02E0002333
:10418C0042F8043B084B9A42F9D301F0A1FD01F02F
:10419C00A3FFFEF7E3FF7047B461000800000020A6
:1041AC00DC030020DC03002088080020FEE7000070
:1041BC00836861F300038360704700BF0023012212
:1041CC00037043708370C270704700BF43680A78F5
:1041DC0062F30823436083684A7862F34103836087
:1041EC0083688A7862F3CB238360CB78C26A013B05
:1041FC0063F31752C2627047836861F308238360CC
:10420C00704700BF836843F008038360704700BFAA
:10421C008068C0F3C0007047836843F00403836078
:10422C00704700BF8068C0F38000704710B411293C
:10423C0017D8DFE811F0120079007E0083008800A7
:10424C008D00920097009C00A100A600AB00B0006E
:10425C00B500BA00BF00C4007400046963F3020423
:10426C000461013A0F2A0DD8DFE802F00E13181D75
:10427C0022272C31363B40454A4F5408C36A61F320
:10428C00D333C36210BC7047436B61F304034363C5
:10429C00F8E7436B61F349134363F3E7436B61F353
:1042AC008E234363EEE7436B61F3D3334363E9E758
:1042BC00436B61F318534363E4E7436B61F35D6352
:1042CC004363DFE7036B61F304030363DAE7036B18
:1042DC0061F349130363D5E7036B61F38E23036327
:1042EC00D0E7036B61F3D3330363CBE7036B61F369
:1042FC0018530363C6E7036B61F35D630363C1E7A4
:10430C00C36A61F30403C362BCE7C36A61F3491374
:10431C00C362B7E7C36A61F38E23C362B2E7C468B2
:10432C0063F35754C4609CE7046963F3C5040461E8
:10433C0097E7046963F38814046192E7046963F3F3
:10434C004B2404618DE7046963F30E34046188E740
:10435C00046963F3D134046183E7046963F394441F
:10436C0004617EE7046963F35754046179E70469D7
:10437C0063F31A64046174E7046963F3DD64046134
:10438C006FE7C46863F30204C4606AE7C46863F34C
:10439C00C504C46065E7C46863F38814C46060E74F
:1043AC00C46863F34B24C4605BE7C46863F30E34E6
:1043BC00C46056E7C46863F3D134C46051E7C46881
:1043CC0063F39444C4604CE7836807298CBF43F0C3
:1043DC0000736FF359638360836861F353438360A5
:1043EC00836862F314538360704700BF024B9A6872
:1043FC0060F3D7529A60704700240140836861F3E0
:10440C0096538360704700BF20B9034BDA6961F3A0
:10441C000002DA61704700BF0000014010B412497D
:10442C000B6843F001030B600B689B07FCD54B68D2
:10443C000D4A6FF301034B60536813F00C0FC3F379
:10444C008101F9D1136823F0867323F48033136050
:10445C0041F610744FF480104FF41F035160D46276
:10446C00106310BC9360704700100240030C03F102
:10447C00804303F5043300F01F001A68012303FA8C
:10448C0000F030EA02030CBF01200020704700BF8F
:10449C00030C03F1804303F5043301291A6800F07F
:1044AC001F0006D0012101FA00F022EA000018607A
:1044BC00704701FA00F0104318607047030C03F1C9
:1044CC00804303F5043301291A6800F01F0006D05D
:1044DC00012101FA00F022EA00001860704701FA8D
:1044EC0000F0104318607047042809D8DFE800F08A
:1044FC00090F151B03000F4B5A6A61F300025A6235
:10450C0070470C4B1A6861F300021A607047094B34
:10451C001A6861F310421A607047064B1A6861F30F
:10452C0018621A607047034B1A6A61F300021A6230
:10453C00704700BF00100240024B5A6860F307122C
:10454C005A60704700100240024B5A6860F30A220E
:10455C005A60704700100240024B5A6860F3CD223B
:10456C005A60704700100240054B5A6860F38F3256
:10457C005A605A68C0F3800060F31C725A6070472E
:10458C0000100240134BA0B95A6860F310428446E5
:10459C005A60104B5A6861F395425A605A68C1F3DD
:1045AC00011060F35E725A60DA6A6CF31A62DA62B6
:1045BC0070475A6842F480325A605A6801280BBF1F
:1045CC006FF3514242F400324FF0020C4FF0000CEA
:1045DC005A60DEE700100240024B5A6860F3010299
:1045EC005A60704700100240024B5868C0F38100BB
:1045FC00704700BF0010024038B53F4D6B6813F098
:10460C000C0F0446C3F3810228D0022A2FD03B4B57
:10461C00236039483A4A41683A4DC1F30311515C61
:10462C00CB4063604168C1F302211144097C23FA39
:10463C0001F1E1604168C1F3C221695CCB40A36028
:10464C0045684168C5F30070C1F3813141EA8001CE
:10465C000A44127EB3FBF2F3236138BD6B6D9805EF
:10466C00D5D52B6B9901D2D5274B2360D1E769683F
:10467C00EB6A002BC1F300411DDAEA6AEB6AC2F364
:10468C00031CEA6AC3F3082302F0070269B36968E2
:10469C001E4811F4003F194908BF08460021A3FB2E
:1046AC00000503FB01F10CFA02F20023FCF786FF74
:1046BC0003462060ADE76B686A6812F0C04FC3F325
:1046CC008343C2F341700CD10F2B0AD0023319B1C2
:1046DC00094A526892030AD50C4800FB03F3236085
:1046EC0097E7013303EB0013F1E70848D7E70348DA
:1046FC0000FB03F323608CE70010024000127A00E9
:10470C006461000874610008006CDC0200093D0063
:10471C00012805D0054B5A6D6FF305125A65704789
:10472C00024A536D43F0300353657047001002404A
:10473C0010B404680C490022C3B26FF30004046087
:10474C00083B026042608260C260A2F13332A2FB7D
:10475C0003231B09486810BC9B000F2202FA03F3C9
:10476C0003434B60704700BF00000240036861F3D5
:10477C0000030360704700BF034B1B68034214BF68
:10478C0001200020704700BF000002400023C0E958
:10479C000033C0E902330382704700BF03684BF655
:1047AC00EF721340036002680B89134303600368C4
:1047BC004A7C62F30D3303600368CA7B62F38B237C
:1047CC00036003688A7B62F30923036003684A7BF6
:1047DC0062F3C713036003680A7B62F386130360FA
:1047EC000A7C036862F345130360D1E9002310B41B
:1047FC004C894460826010BCC3607047014BD86028
:10480C00704700BF00200240024B0349034A596025
:10481C005A6070470020024023016745AB89EFCDF9
:10482C00024A136943F08003136170470020024071
:10483C001B4A136943F0020313615061136943F07F
:10484C0040031361D368D90704D4D3685B0720D520
:10485C00012011E04FF08043D168C80712D4D16811
:10486C00490713D4D268D20603F1FF334CBF0220A0
:10487C000320002B08BF0420094B1A696FF3410277
:10488C001A617047013BE7D10420F5E7013B012099
:10489C00EFE7D36813F0100F14BF02200320EBE7EF
:1048AC0000200240194A136943F0010313610160AF
:1048BC00D368D90704D4D3685B0720D5012011E055
:1048CC004FF48013D168C80712D4D168490713D4A8
:1048DC00D268D20603F1FF334CBF02200320002B19
:1048EC0008BF0420094B1A696FF300021A61704764
:1048FC00013BE7D10420F5E7013B0120EFE7D3684A
:10490C0013F0100F14BF02200320EBE7002002402D
:10491C000B88002B43D02DE9F0434FF0000E0326FB
:10492C0001251FFA8EFC4FEA4C0213F0010F06FA18
:10493C0002F705FA0CF80EF1010E2CD0046824EAEB
:10494C00070404608C79D0F80090944044EA090480
:10495C000460446824EA080444600C79D0F80480AC
:10496C0004FA0CFC4CEA08044460846824EA07044A
:10497C008460CC79D0F808C0944044EA0C0484607C
:10498C00C46824EA0707C76091F805C0C4680CFA2C
:10499C0002F22243C2605B08C3D1BDE8F0837047CA
:1049AC0001F007039B00C90802FA03F20BD0416A1D
:1049BC004FF00F0C0CFA03F321EA03034362436A32
:1049CC001A4342627047016A4FF00F0C0CFA03F362
:1049DC0021EA03030362036A1A430262704700BFB1
:1049EC001F4BDB68C3F3022300B5C3F1070EBEF106
:1049FC00040F03F1040C28BF4FF0040EBCF1060F9A
:104A0C0021D9033B4FF0FF3C0CFA03FC22EA0C02C9
:104A1C004FF0FF3C0CFA0EFC21EA0C0199400028E7
:104A2C0041EA020112DB0F4A09011318C9B283F8DB
:104A3C0000130123410900F01F0003FA00F042F8B3
:104A4C0021005DF804FB00221346E1E7064B00F061
:104A5C000F0009010344C9B219765DF804FB00BFCD
:104A6C0000ED00E000E100E0FCEC00E008B52E4BAE
:104A7C0098421CD02D4B984223D02D4B98422AD0D3
:104A8C002C4B984209D02C4B98422ED02B4B984251
:104A9C0035D02B4B98423CD008BD2A480121FFF75A
:104AAC000DFDBDE8084027480021FFF707BD26484B
:104ABC000121FFF703FDBDE8084023480021FFF763
:104ACC00FDBC22480121FFF7F9FCBDE808401F4856
:104ADC000021FFF7F3BC1E480121FFF7EFFCBDE8F6
:104AEC0008401B480021FFF7E9BC1A480121FFF7D9
:104AFC00E5FCBDE8084017480021FFF7DFBC16486D
:104B0C000121FFF7DBFCBDE8084013480021FFF74B
:104B1C00D5BC12480121FFF7D1FCBDE808400F4875
:104B2C000021FFF7CBBC00BF002C0140000400406B
:104B3C0000100040002000400040014000440140B3
:104B4C0000480140080010000B000C000100100090
:104B5C000400100010000C0011000C0012000C00DE
:104B6C00036861F3C7130360704700BF062909D8B7
:104B7C00DFE801F013080E0809080400C36962F3AA
:104B8C00CB23C3617047C36962F3C303C36170472E
:104B9C00836962F3CB2383617047836962F3C30338
:104BAC0083617047062909D8DFE801F0090E131854
:104BBC001D220400036A62F30C3303627047036A1C
:104BCC0062F3000303627047036A62F382030362B9
:104BDC007047036A62F3041303627047036A62F35B
:104BEC00861303627047036A62F3082303627047FB
:104BFC00036A62F38A230362704700BF2DE9F04118
:104C0C0086B0054601A817461E468846FFF7F4FCF9
:104C1C00DDE90334114A954208BF1C4604EB8404B9
:104C2C006400B4FBF8F10E4CA4FB0134E40804EB73
:104C3C008403A1EB43010429AB6888BF0134A4B2FF
:104C4C0064F30F03AB60EB6867F30C33EB602B6919
:104C5C0066F30D332B6106B0BDE8F08100380140DE
:104C6C00CDCCCCCCC36861F34D33C360704700BF6F
:104C7C00C36861F3C303C360704700BFC36861F3CB
:104C8C008203C360704700BF436961F3C71343617C
:104C9C00704700BF436961F3C3034361704700BFB2
:104CAC00064B0748B3F804C00649074AA0F800C0F1
:104CBC0018885B8808801380704700BF5407002059
:104CCC00F2060020F60600206C06002030B54023CA
:104CDC0087B0002203214FF09040FCF709FF082316
:104CEC00002203214FF09040FCF702FF01214FF40A
:104CFC00A010FFF7CDFB3448344CFFF719FD01A889
:104D0C00FFF744FD324B334A2F48019301A940F27F
:104D1C0001234FF440350492ADF81430CDE902452F
:104D2C00FFF73CFD28480121FFF720FD01212A480F
:104D3C00FFF7AEFB0720FFF717FC6846FFF73EFABC
:104D4C0001240325002325488DF8023069468DF88F
:104D5C0000408DF801408DF80350FFF737FA1F48DB
:104D6C002B4622462946FFF761FA1C482B460621A2
:104D7C000222FFF75BFA2B462A4610211748FFF751
:104D8C0055FA2046FFF732FB224614480721FFF75D
:104D9C001BFB12482146FFF72FFA10482146FFF75C
:104DAC0007FA0E48FFF72EFA0C48FFF731FA0028E5
:104DBC00FAD10A48094CFFF72FFA2046FFF732FACE
:104DCC000028FAD107B030BD08000240540700207B
:104DDC004C2401400001010109001800002401408D
:104DEC0048F2E80300FB03F3002BB8BF03F6FF7394
:104DFC00064A43F23810A0EB233082FB0023C01785
:104E0C00A0EBE3000F3000B2704700BF310CC33091
:104E1C00FEE700BFFEE700BFFEE700BFFEE700BFF6
:104E2C00704700BF704700BF704700BF704700BF9E
:104E3C0010B50220FFF7A0FC012800D010BD054CD6
:104E4C006060FFF72DFF0820FFF796FC012808BFD4
:104E5C00606010BD0000024008B52020FFF78CFCFC
:104E6C00012806D10A4B10225A60DA696FF300024E
:104E7C00DA618020FFF780FC012800D008BD044BCC
:104E8C0010225A60DA696FF30002DA6108BD00BFC4
:104E9C000000024008B5264B1B78002B39D14FF48B
:104EAC008040FFF769FC012811D04FF40050FFF748
:104EBC0063FC01281ED04FF40040FFF75DFC012875
:104ECC0000D008BD1B4B4FF480525A6008BD1A4BE2
:104EDC001B78002BE9D0194A1649136A4FF480400D
:104EEC0043F00203136248604FF40050FFF744FC98
:104EFC000128E0D10F4B4FF480525A605A6C6FF37B
:104F0C0000025A64FEF79AFE0D4B4FF400421A61F0
:104F1C00D1E7084B4FF480525A605A6C6FF3000281
:104F2C005A64FEF78BFE064B4FF400421A6108BD23
:104F3C009605002000000240970500200004004068
:104F4C0000040140084B5A69920209D50749084AE6
:104F5C004FF4001058614B6A1268B3EB520F00D833
:104F6C007047FDF765B900BF000401400010004018
:104F7C006C000020024B4FF6FE721A61FDF7E0BE8A
:104F8C0000200040024B00221A61FDF713B900BF4C
:104F9C0000440140034B4FF6FE714FF6FD72196150
:104FAC001A61704700400140704700BF074B1A69F7
:104FBC00910744BF4FF6FD721A61044B1A69D20770
:104FCC0044BF4FF6FE721A61704700BF00040040E8
:104FDC00064A07491368013313604B691B0400D45C
:104FEC0070474FF400434B61FDF794BD5C07002004
:104FFC0000040140024BD869C0F38070704700BFB9
:10500C0000000140044B1A684FF4001122F4001206
:10501C001A605961704700BF00040140024A1368CE
:10502C0043F400131360704700040140054B064A1B
:10503C001B78002B0CBF4FF4001100215B05916015
:10504C00D360704765000020000401402DE9F04357
:10505C000029B4BFCE1C0E4626F00303073383B0E1
:10506C0023F0070300AFADEB030DB6106D46884679
:10507C008146144600213246284601F051F8B8F119
:10508C00030F17DD4846291F0022837890F8038010
:10509C0090F800E090F801C01B0443EA086343EA6F
:1050AC000E03013243EA0C23964241F8043F00F10F
:1050BC000400EADC3E60FFF7A7FBC4F30903EBB185
:1050CC0000237B607B683A689A4211D978687B68C8
:1050DC0004EB800055F82310FFF7E4FB0320FFF7E7
:1050EC008DFB7B6801337B607A683B689A42EDD319
:1050FC00FFF796FB0C37BD46BDE8F0832046FFF763
:10510C0097FBDDE7002A09DD431E013103EB020C9E
:10511C00081AC25C03F8012F6345FAD1704700BF2F
:10512C0038B5164D164C6B6C6B642046FFF79EFC25
:10513C00144B41210B22A16122621A78A2624FF614
:10514C00FF73E3626269104B002142F0010262615D
:10515C0003F8041B0D4A6162EA640D4A2B6513784F
:10516C00AB64E36843F40073E360236843F001032A
:10517C0040F68B1223606A6438BD00BF0000024009
:10518C0000040040D20300206007002034040040DB
:10519C00CE03002038B51D4D1D4C6B6C43F0100335
:1051AC006B642046FFF762FC60210323194AA1615E
:1051BC0023621278184BA2624C210122E1621A7010
:1051CC0063691649164A43F001036361154BE964A0
:1051DC002A655B781733AB646B6C43F002036B642A
:1051EC006B6C43F008036B646B6C43F001036B64F2
:1051FC00E36843F40073E360636C43F4004363645B
:10520C00236843F00103236038BD00BF0000024057
:10521C0000040040440700206007002034040040D4
:10522C003C040020D2030020024B186900F010004F
:10523C00704700BF000400480248102301220221DD
:10524C00FCF762BC0004004862B670471C4B40F28D
:10525C00531210B51A60FFF7E1F801210020FFF797
:10526C0043F90120FFF702F901280446F9D1002087
:10527C001D21FFF787F921460220FFF735F9192088
:10528C00FFF7F4F801280446F9D10020FFF754F990
:10529C000020FFF761F90020FFF756F92046FFF7D1
:1052AC0037FA0220FFF798F9FFF79EF90228FBD195
:1052BC000020FFF72DFABDE8104000F039BD00BF0B
:1052CC000020024008B511480121FFF7E1F8012147
:1052DC004FF4C010FFF7DCF80223002203214FF03B
:1052EC009040FCF705FC2023002203214FF0904056
:1052FC00FCF7FEFB064B002083F80C034FF48052A6
:10530C001A600121BDE80840FFF77EB811001400B7
:10531C0000E100E0084B10B44CF6CC4245F2555479
:10532C001C6003201A604FF47A614AF6AA22586076
:10533C0010BC99601A6070470030004038B53F4887
:10534C003F4C0121FFF7A4F80025682340F6B83143
:10535C0046F66802E1622046A5622946A261E36135
:10536C000122FFF703FC204601220221FFF7FEFB7E
:10537C00012220460421FFF7F9FB20460121FFF70B
:10538C00EFFB636C2F48502262F307036364012127
:10539C00FFF77EF82C4C2D480121FFF779F80223FA
:1053AC0019462A462046FCF7A3FB2A462046012331
:1053BC000221FCF79DFB80232A4602214FF09040EE
:1053CC00FCF796FB204602220121FFF7E9FA294659
:1053DC0020460222FFF7E4FA022207214FF0904008
:1053EC00FFF7DEFA2A464FF4806302214FF090401B
:1053FC00FCF77EFB2A464FF4007302214FF09040DD
:10540C00FCF776FB4FF480732A4602214FF0904054
:10541C00FCF76EFB02220A214FF09040FFF7C0FA16
:10542C00022209214FF09040FFF7BAFABDE838404C
:10543C00022208214FF09040FFF7B2BA0B0018007F
:10544C00002C01401100140000040048120014004C
:10545C0010B51948194C0121FFF71AF81848012109
:10546C00FFF716F81023204600220221FCF740FB20
:10547C00012220460421FFF793FA01214FF4A010DA
:10548C00FFF706F80F49104B40F68A1010224864BB
:10549C0083F80B234FF4006119600C4B4FF6FF712E
:1054AC00D9629A621A6842F080021A601A6842F055
:1054BC0001021A6010BD00BF120014000004004865
:1054CC0001001C000000024000E100E0000400406C
:1054DC0070B5FFF7BBFE264C01214FF4A010FEF770
:1054EC00D7FF102384F80B334FF400632360FFF7CE
:1054FC0025FF20480121FEF7CBFF1F4B1F484FF61D
:10550C00FF763B25DE6201219D62FEF7C1FF1C4B3D
:10551C003222DA6277229A62302384F813334FF402
:10552C0000232360FFF7CEFE16480121FEF7B0FFE3
:10553C00154B1648DE629D621A6842F080021A60B2
:10554C000121FEF7A5FF124B4FF4FA72DA629D624D
:10555C001A68002142F080021A6084F815134FF487
:10556C0000132360FFF774FFBDE8704000F036BBFA
:10557C0000E100E004001C000010004008001C00CA
:10558C0000200040120018000048014011001800D3
:10559C0000440140014B5863704700BF002C014090
:1055AC00014B9863704700BF002C0140014BD8633E
:1055BC00704700BF002C0140024A536943F00103BD
:1055CC0053617047002C0140024B0022DA625A6290
:1055DC00704700BF0004004010B5384C0122204633
:1055EC000021FFF7DFFA204601220221FFF7DAFA49
:1055FC00204601220421FFF7D5FA0122114620464C
:10560C00FFF7D0FA204601220321FFF7CBFA204600
:10561C0001220521FFF7C6FA2268294B294842F0DE
:10562C0001022260626C42F400426264626942F0E0
:10563C00010262611968244A41F00101196059693B
:10564C0041F001015961D96821F00101D96001686B
:10565C0041F001010160116841F0010111605169D3
:10566C00A3F5923341F0010151611A6842F0010235
:10567C001A605A6942F001025A61DA6842F001027A
:10568C00A4F59434DA60FFF721FB012200212046B7
:10569C00FFF788FA23680D4A43F0010320212360A9
:1056AC0082F807138023136002F1C04202F50C52FA
:1056BC00136843F40043136010BD00BF002C01407D
:1056CC0000440140004801400010004000E100E0AF
:1056DC0070B54FF0904420464FF4806300220121B6
:1056EC00FCF706FA4FF48060A0624FF4007320467A
:1056FC0000220121FCF7FCF94FF400700F4DA06261
:10570C004FF48073204600220121FCF7F1F90223AB
:10571C004FF480701946A06200222846FCF7E8F985
:10572C002846012300220221FCF7E2F920468023BF
:10573C00BDE8704000220221FCF7DAB900040048F1
:10574C0010B50E4B1A788AB90D4C01231946204618
:10575C00FCF7CEF90123A362BDE810404FF40073AF
:10576C00002202214FF09040FCF7C2B904480123FB
:10577C0000220221FCF7BCF9EEE700BF0400002078
:10578C000004004810B50F4B1A78802392B9012100
:10579C004FF09040FCF7ACF94FF0904380229A62A6
:1057AC00BDE810404FF48073002202214FF090406E
:1057BC00FCF79EB9002202214FF09040FCF798F9BB
:1057CC00EEE700BF0400002010B50E4B1A788AB922
:1057DC000D4C022301212046FCF78AF90223A36217
:1057EC00BDE810404FF48063002202214FF090403E
:1057FC00FCF77EB90223044800221946FCF778F91D
:10580C00EEE700BF040000200004004870B51D4EF8
:10581C0002230022012130464FF09044FCF768F936
:10582C0002204FF4806300220121B0622046FCF775
:10583C005FF901234FF480601D4619460022A062D7
:10584C003046FCF755F94FF40073002229462046E8
:10585C00B562FCF74DF94FF4007180230022A16270
:10586C0020462946FCF744F98023A36200224FF41A
:10587C00807329462046FCF73BF94FF48073A362F2
:10588C0070BD00BF00040048013870B5052833D83E
:10589C00DFE810F033005F008B00B800E500060075
:1058AC00854C01231D46194620460022FCF720F9A1
:1058BC00A5624FF090444FF4007300222946204615
:1058CC00FCF716F94FF4007180230022A1622046E8
:1058DC002946FCF70DF9802000224FF480732946ED
:1058EC00A0612046FCF704F94FF48073A362FFF724
:1058FC006BFF724B724ADA6170BD4FF0904480239B
:10590C00002201212046FCF7F3F880206A4DA062AA
:10591C004FF48073002201212046FCF7E9F80123A3
:10592C004FF4807019460022A0622846FCF7E0F87C
:10593C00012100224FF40073A9612046FCF7D8F82E
:10594C004FF40073A362FFF73FFF5C4B5D4ADA61D3
:10595C0070BD594C0223002201212046FCF7C8F8E7
:10596C004FF0904502204FF4806300220121A06289
:10597C002846FCF7BDF801234FF48060194600223D
:10598C00A8622046FCF7B4F8012100224FF4007302
:10599C00A1612846FCF7ACF84FF40073AB62FFF73B
:1059AC00F1FE464B484ADA6170BD434C01231D465B
:1059BC004FF09046194600222046FCF799F84FF418
:1059CC000073002229463046A562FCF791F84FF48B
:1059DC0000720223B262294600222046FCF788F8A6
:1059EC0002224FF480632946A26130460022FCF764
:1059FC007FF84FF48063B362FFF7C4FE2F4B304A3D
:105A0C00DA6170BD4FF090448023002201212046C2
:105A1C00FCF76EF88020284DA0624FF480730022B2
:105A2C0001212046FCF764F84FF480710223002218
:105A3C00A16228460121FCF75BF8022100224FF4F9
:105A4C008063A96120460121FCF752F84FF4806372
:105A5C00A362FFF775FE194B1A4ADA6170BD164D39
:105A6C000223002201212846FCF742F84FF0904413
:105A7C0002214FF480630022A96220460121FCF729
:105A8C0037F84FF48060802300220121A062204669
:105A9C00FCF72EF8802000224FF480730121A061C6
:105AAC002046FCF725F84FF48073A362FFF748FEFD
:105ABC00024B054ADA6170BD000400480000014049
:105ACC00C1000040E1000040D100004070B51D4E07
:105ADC0002230022012130464FF09044FCF708F8D5
:105AEC0002204FF4806300220121B0612046FBF7B5
:105AFC00FFFF01234FF480601D4619460022A0626F
:105B0C003046FBF7F5FF4FF4007300222946204680
:105B1C00B561FBF7EDFF4FF4007180230022A16209
:105B2C0020462946FBF7E4FF8023A36100224FF4B3
:105B3C00807329462046FBF7DBFF4FF48073A3628A
:105B4C0070BD00BF0004004808B5FFF73DFEFFF72D
:105B5C00F7FDBDE80840FFF715BE00BF044A054B32
:105B6C0012781A62DA6942F00102DA61704700BFFA
:105B7C00D40300200000024010B5174CBDF808C03B
:105B8C002271120AE2701A0AA1706271090A4FEAB4
:105B9C001C22617084F808C02070A371E271A446C5
:105BAC0004F1080E0021414008224B0011F0800F37
:105BBC0083F0070314BFD9B2490002F1FF3308BFC9
:105BCC00C9B213F0FF02F0D1F44502D01CF8010F5A
:105BDC00E9E7617210BD00BF6408002030B532489F
:105BEC00324D334C89B00121FEF752FC3148012172
:105BFC00FEF74EFC01214FF4A010FEF749FC2E4B92
:105C0C0001A928464022CDE90123FEF781FE00229E
:105C1C0006212846FEF7C4FE2046FEF789FD03A8A0
:105C2C00FEF7B4FD254B1A78254BADF81620002550
:105C3C00244A049303A920464FF480731024ADF832
:105C4C00144003920693ADF81C50FEF7A7FD1E4AB4
:105C5C001E4CD16941F00201D161D16941F00801BA
:105C6C002B46D16120462A464FF4E131FEF7C6FFA0
:105C7C0020460121FEF7FCFF20460121FEF7FEFF26
:105C8C0020460121FFF706F820460121FEF7FCFF14
:105C9C0020460121FEF7E6FF2A4603210A20FEF7E3
:105CAC009FFE09B030BD00BF0E0018000004004874
:105CBC001C0002401200140000010201D403002059
:105CCC006408002004380140000002400038014004
:105CDC0030B414490B6843F001030B600B689B074D
:105CEC00FCD54B680F4A6FF301034B60536813F0FC
:105CFC000C0FC3F38101F9D113680B480B4C23F043
:105D0C00867323F48033136041F610754FF48013BF
:105D1C005160D56213634FF41F039360846030BCF1
:105D2C00704700BF0010024000ED00E000100008BA
:105D3C0010B5FEF759FC60B1022816D02C482D4B3B
:105D4C002D495B682D4AC3F30313CB5CD84010601C
:105D5C0010BD284B5A6D9205F0D51A6B244B284870
:105D6C0012F0007F08BF1846E9E7224B5968DA6A3F
:105D7C00002AC1F300411CDAD86ADC6ADA6AC0F383
:105D8C00031EC4F3082402F0070259B35B681D48D4
:105D9C0013F4003F164B4FF0000108BF18460EFAE3
:105DAC0002F20023A4FB000E04FB01F1FBF706FC3E
:105DBC00C5E758685B6813F0C04FC0F38340C3F36A
:105DCC0041720BD10F2809D0023019B1094B5B6815
:105DDC009B0309D50B4B03FB00F0B0E7013000EB44
:105DEC000210F2E70748DAE7014B03FB00F0A6E7E5
:105DFC0000127A000010024084610008D8030020D1
:105E0C00006CDC0200093D002DE9F047089E0D46B0
:105E1C0004468846002B4DD18A42944668D9B2FA82
:105E2C0082F252B101FA02F3C2F1200120FA01F11F
:105E3C000CFA02FC41EA030894404FEA1C45210C81
:105E4C00B8FBF5FE1FFA8CF705FB1E8341EA0343F2
:105E5C000EFB07F199420BD91CEB03030EF1FF303B
:105E6C0080F01E81994240F21B81AEF1020E634418
:105E7C005B1AA4B2B3FBF5F005FB103344EA034400
:105E8C0000FB07F7A7420AD91CEB040400F1FF330F
:105E9C0080F00881A74240F2058164440238E41B7B
:105EAC0040EA0E4000211EB1D4400023C6E9004355
:105EBC00BDE8F0878B4208D9002E00F0EE8000215F
:105ECC00C6E900050846BDE8F087B3FA83F100295E
:105EDC004AD1AB4202D3824200F2F980841A65EBBC
:105EEC00030301209846002EE2D0C6E90048DFE704
:105EFC0002B9FFDEB2FA82F2002A40F09180A1EBE7
:105F0C000C054FEA1C471FFA8CFE0121B5FBF7F379
:105F1C0007FB1350250C45EA00450EFB03F0A84285
:105F2C0008D91CEB050503F1FF3802D2A84200F298
:105F3C00CB8043462D1AA4B2B5FBF7F007FB1055E6
:105F4C0044EA05440EFB00FEA64508D91CEB0404EC
:105F5C0000F1FF3502D2A64500F2BB802846A4EB27
:105F6C000E0440EA03409EE7C1F120078B4022FA61
:105F7C0007FC4CEA030C20FA07F405FA01F31C4366
:105F8C00FD404FEA1C4900FA01F3B5FBF9F8200C6F
:105F9C001FFA8CFE09FB185540EA054508FB0EF06C
:105FAC00A84202FA01F20BD91CEB050508F1FF3AE5
:105FBC0080F08880A84240F28580A8F102086544F0
:105FCC002D1AA4B2B5FBF9F009FB105544EA0545AE
:105FDC0000FB0EFEAE4508D91CEB050500F1FF34A5
:105FEC006CD2AE456AD90238654440EA0840A0FB41
:105FFC000294A5EB0E05A542C846A64656D353D02F
:10600C005EB1B3EB080265EB0E0505FA07F722FA51
:10601C0001F3CD401F43C6E900750021BDE8F087B0
:10602C00C2F1200320FA03F10CFA02FC25FA03F367
:10603C0095400D434FEA1C471FFA8CFEB3FBF7F15A
:10604C0007FB11302B0C43EA004301FB0EF0984286
:10605C0004FA02F408D91CEB030301F1FF382FD228
:10606C0098422DD9023963441B1AADB2B3FBF7F039
:10607C0007FB103345EA034500FB0EF3AB4208D98E
:10608C001CEB050500F1FF3816D2AB4214D90238CF
:10609C006544ED1A40EA014138E73146304607E7DE
:1060AC008646E5E61846FAE64B45A9D2B9EB020856
:1060BC0064EB0C0E0138A3E74046EAE7204694E770
:1060CC004146D1E7D0467BE7023B654432E70846C0
:1060DC0009E76444023842E770B50D4D0D4C641B62
:1060EC00A4100026A64209D10B4D0C4C00F020F850
:1060FC00641BA4100026A64205D170BD55F8043BC4
:10610C0098470136EEE755F8043B98470136F2E71D
:10611C00AC610008AC610008AC610008B06100081B
:10612C0002440346934200D1704703F8011BF9E780
:10613C00F8B500BFF8BC08BC9E467047F8B500BF68
:08614C00F8BC08BC9E46704738
:10615400191B12131D1516171A090A0B1E0D0E0F03
:106164000000000000000000010203040607080903
:10617400000000000102030402040608020C0810D7
:1061840000000000000000000102030406070809E3
:1061940041545F46345F345F4634323100000000BE
:0861A40070FCFF7F0100000008
:0461AC0021160008B0
:0461B000FD150008D1
:1061B400007C000801010102881388137800500054
:1061C4005000D0070E004C046C07DC0564004A0143
:1061D400050A0A509001C800FF00CA000501140016
:1061E4004600DC05E8030000102700000000000062
:1061F4000A0000000000000064000000000000002D
:106204000000000000000000000000001027000053
:10621400FF0700000301050101010000D430000064
:106224000105010AB400D007D0070000B400B7008C
:10623400BA00BD00C100C400C700CA00CD00D00030
:10624400D300D600D900DC00E000E300E600E9005A
:10625400EC00EF00F200F500F700FA00FD00000189
:106264000301060109010B010E01110113011601BD
:1062740019011B011E0120012301250128012A0106
:106284002C012F0131013301350138013A013C0160
:106294003E014001420144014601470149014B01CD
:1062A4004D014E0150015101530154015601570152
:1062B40058015A015B015C015D015E015F016001EF
:1062C40061016201630163016401650165016601A5
:1062D4006601670167016701680168016801680177
:1062E4006801680168016801680167016701670165
:1062F4006601660165016501640163016301620170
:10630400610160015F015E015D015C015B015A0195
:1063140058015701560154015301510150014E01D6
:106324004D014B014901470146014401420140012D
:106334003E013C013A0138013501330131012F019D
:106344002C012A0128012501230120011E011B0122
:1063540019011601130111010E010B0109010601B6
:1063640003010001FD00FA00F700F500F200EF0060
:10637400EC00E900E600E300E000DC00D900D60010
:10638400D300D000CD00CA00C700C400C100BD00C6
:10639400BA00B700B400B100AE00AB00A700A4007F
:1063A400A1009E009B009800950092008F008C0035
:1063B4008800850082007F007C00790076007300ED
:1063C40071006E006B006800650062005F005D0094
:1063D4005A005700550052004F004D004A00480033
:1063E4004500430040003E003C00390037003500C2
:1063F400330030002E002C002A0028002600240040
:10640400220021001F001D001B001A0018001700A5
:10641400150014001200110010000E000D000C00F5
:106424000B000A000900080007000600050005002B
:106434000400030003000200020001000100010047
:106444000000000000000000000000000000000048
:10645400000001000100010002000200030003002B
:1064640004000500050006000700080009000A00F2
:106474000B000C000D000E0010001100120014009F
:106484001500170018001A001B001D001F00210032
:1064940022002400260028002A002C002E003000B0
:1064A40033003500370039003C003E004000430013
:1064B400450048004A004D004F0052005500570067
:1064C4005A005D005F006200650068006B006E00AA
:1064D40071007300760079007C007F0082008500E3
:1064E40088008C008F009200950098009B009E000D
:1064F400A100A400A700AB00AE00B10050001E0331
:1065040003000000000000009001000000000000F3
:10651400E80300000000000000000000000000008C
:1065240000000000204E0000A08601006419000055
:106534000000000001000000000000003200000024
:106544000000000000000000000000000000000047
:106554001027000050C30000010201006E00D007A4
:1065640064000500E8030614320078004B005A006A
:106574005A001E0002010000FA000000204E200014
:0C65840050C311070A00000000127A004A
:107BE00041545F46345F30345F4634323100000028
:107BF0000000000000000000000000000000000085
:04000005080041713D
:00000001FF
